:100000000C9457010C9474010C9474010C947401B9
:100010000C9474010C9474010C9474010C9474018C
:100020000C9474010C9474010C94D01C0C94A21DBB
:100030000C94D7170C9474010C9474010C947401F3
:100040000C9474010C9474010C9474010C9474015C
:100050000C9474010C945F180C9474010C9474014A
:100060000C9474010C9474010C9474010C9474013C
:100070000C9474010C9474010C9474010C9474012C
:100080000C9474010C9474010C9474010C9474011C
:100090000C9474010C9474010C9474010C9474010C
:1000A0000C9474010C9474010C94740124042404C1
:1000B00050045004B204D004E805E805DB047405DC
:1000C000850585050F1E361E2E1F361E2E1F821E0D
:1000D000A51E2E1FFC1E0B1F14001A000800150081
:1000E00017000000000000000000000004001600DF
:1000F000070009000A0000000000000000000000E6
:100100001D001B0006001900050000000000000093
:10011000000000000000000029002C002B0000005F
:1001200000000000000000000000000000000000CF
:1001300000001C0018000C0012001300000000005A
:100140000000000000000B000D000E000F002E004C
:100150000000000000000000000011001000360048
:1001600037002D0000000000000000000000280003
:100170002A00005C000000000C0362006F006C00AD
:1001800065006B0000001C034D0069006B006F00F0
:10019000420161006A0020004200690065006C00B5
:1001A00000000403090409023B00020100A0FA094F
:1001B0000400000103010100092111010001224096
:1001C0000007058103080001090401000103000084
:1001D00000092111010001227B0007058203200094
:1001E000011201000200000008EDFE0837010001C5
:1001F00002000105010902A10185020901A1000512
:1002000009190129081500250195087501810205C4
:1002100001093009311581257F950275088106098C
:10022000381581257F950175088106050C0A38026D
:100230001581257F950175088106C0C005010980DB
:10024000A101850319012AB700150126B700950100
:1002500075108100C0050C0901A101850419012A4E
:10026000A002150126A002950175108100C00501AC
:100270000906A101050719E029E7150025019508E0
:10028000750181029501750881010507190029FF93
:10029000150026FF0095067508810005081901293B
:1002A00005950575019102950175039101C0112411
:1002B0001FBECFEFDAE0DEBFCDBF11E0A0E0B1E0BE
:1002C000E2ECFFE302C005900D92AE38B107D9F71A
:1002D00022E0AEE8B1E001C01D92AD38B207E1F70F
:1002E0000E9420120C94DF1F0C94000081E00895FE
:1002F00081E008950C94780108950C947C011F937B
:10030000CF93DF9300D000D01F92CDB7DEB74983E3
:100310005A836B833091910189819A81311114C084
:10032000662359F0222349F00E942508182F682FD0
:1003300089819A810E94CE0703C00E94F907182F75
:1003400069817A81812F04C00E94250869817A81A0
:100350000F900F900F900F900F90DF91CF911F9102
:100360000C948B0FFC01262F408151816281738197
:1003700084810C947F0181E00895CF93DF93EC0199
:1003800060E00E94B201BE01DF91CF910C947D012B
:100390000C94D1100C94CD1008950E9478060E9400
:1003A000CC012FEF84E39CE0215080409040E1F7A6
:1003B00000C000000C9485180F931F93CF93DF9318
:1003C0008C0161E00E94B201EC01B8010E947A0147
:1003D0008823F1F1B801CE010E94A2168823C1F151
:1003E000B801CE010E94B614882391F1B801CE0164
:1003F0000E94FE15882361F1F8018281882309F1AA
:10040000CB358DE5D807C1F050F4C115FCE5DF0709
:1004100081F0CF3DDC45A9F40E948C0D19C0CC358C
:10042000EDE5DE0761F0CD35DD4559F40E94CF0CD6
:1004300008C00E94CD010CC00E94D80C02C00E94CE
:10044000DB0CC801DF91CF911F910F910C947601C5
:1004500080E0DF91CF911F910F9108950E94B9170D
:100460000C9447020E944A020C94BF1708950C9402
:10047000360281E008950C9439020895CF93C82F75
:100480000E9437028C2F0E943B02CF91089580E09A
:100490000C943E020E94FE160C943E020E94FE1630
:1004A00090919001891721F0809390010C943E0265
:1004B0000895CF93DF93CDB7DEB72B970FB6F8949F
:1004C000DEBF0FBECDBF4F83588769877A878B8782
:1004D00061110E941B0C9E012F5F3F4F86E0F901C6
:1004E00011928A95E9F785E0FE013796D9010190CE
:1004F0000D928A95E1F789819A814C815D81452B26
:1005000031F09F3F31F491E08F3F19F403C091E047
:1005100001C090E090FF09C049815A816B817C81C4
:100520008D819E810E943C0B05C0C9010E94BB01C8
:100530008111F2CF2B960FB6F894DEBF0FBECDBF60
:10054000DF91CF910895FC01808191810E9467081D
:100550000895CF93882309F4A4C0C82F8238C1F42A
:100560000E94FE1681FD9DC069E380910201909179
:1005700003010E9491170E943D0C2FEF81EE94E041
:10058000215080409040E1F700C0000069E319C0AD
:10059000833801F50E94FE1680FD83C063E58091DB
:1005A0000201909103010E9491170E943D0C2FEFD0
:1005B00081EE94E0215080409040E1F700C00000BF
:1005C00063E580910201909103010E949317CF91FE
:1005D0000C943D0C8438C1F40E94FE1682FD61C06B
:1005E00067E480910201909103010E9491170E949B
:1005F0003D0C2FEF81EE94E0215080409040E1F7D8
:1006000000C0000067E4DDCF8CEF8C0F813AD0F49E
:100610006C2F80910201909103010E945B17882347
:1006200049F06C2F80910201909103010E94931771
:100630000E943D0C6C2F80910201909103010E9459
:100640009117C5CF80E28C0F883048F4C77081E0E5
:1006500001C0880FCA95EAF70E94FE0BB8CFEBE500
:10066000EC0FE33040F4F0E0E95BFE4F808190E076
:10067000CF910C942317E8E5EC0FE73150F4F0E04C
:10068000EE0FFF1FE75EFE4F80819181CF910C94AA
:100690003917CD3E30F08C2F0E94A512CF910C94CB
:1006A0007713CF910895882309F464C0823879F4D0
:1006B0000E94FE1681FF5EC069E380910201909165
:1006C00003010E9491170E943D0C69E310C083381A
:1006D000B1F40E94FE1680FF4DC063E580910201D7
:1006E000909103010E9491170E943D0C63E5809157
:1006F0000201909103010E9493170C943D0C8438E1
:1007000079F40E94FE1682FF35C067E480910201F1
:10071000909103010E9491170E943D0C67E4E7CF7E
:100720009CEF980F913A10F4682FE1CF90E2980F68
:10073000983050F4877091E001C0990F8A95EAF7DC
:10074000892F0E94040CD9CF9BE5980F933020F499
:1007500080E090E00C94231798E5980F973120F4EF
:1007600080E090E00C9439178D3E20F00E94001339
:100770000C94771308951F93CF93DF93182FEB01F9
:100780000E94A902209741F08FE99FE00197F1F7BD
:1007900000C000002197F6CF812FDF91CF911F91EC
:1007A0000C945303893319F060E070E002C060E5F7
:1007B00070E00C94BB03882321F00E94FE0B0C9484
:1007C0003D0C0895882321F00E94040C0C943D0CEC
:1007D0000895CF92DF92EF92FF920F931F93CF93E2
:1007E000DF937C01D62FC72FFC0112810581029572
:1007F0000F700E94F40B8823B9F01123A9F08C2FFD
:10080000807F803421F080E28D0F883068F0809105
:100810005B0282FD09C082E00E949D0C0E94F40BE5
:1008200091E0D82ED92601C0D12CCC2EC2948FE0D5
:10083000C8228C2D90E08C30910508F0C9C1FC01D4
:10084000EA5AFF4F0C94761F8C2F807FCF7088233D
:1008500011F0C295C07F112399F0CC2309F4A4C1F3
:1008600080E28D0F883010F0D11104C08C2F0E94CF
:10087000FE0B03C08C2F0E940E0C0E943D0C94C1F5
:100880008D2F0E945303CC2309F4A2C180E28D0F67
:10089000883038F1DD2329F18C2F0E94140C24C0FC
:1008A0008C2F807FCF70803211F0C295C07FDD2306
:1008B00019F0D130A1F140C080915B0282FF17C0D6
:1008C000112349F0CC2329F08C2F0E94FE0B0E94AB
:1008D0003D0C80E06AC180E00E945303CC2309F400
:1008E00077C18C2F0E94040C0E943D0C71C1112312
:1008F00071F0002341F0013031F40E941E0C8C2B6A
:100900000E94260C65C10E941E0C8C2B0EC0002379
:1009100019F0013009F45CC10E94330C1FC011238F
:1009200039F0063008F054C18C2F0E94DB0350C10F
:10093000053008F04DC112C0112319F00023A1F3B6
:1009400033C1002359F0D93309F03FC1FFEF07EE5F
:1009500013E0F15000401040E1F735C18C2F0E94A8
:10096000E20336C18C2F86958695837019F081300D
:1009700061F02EC1112321F08D2F9C2F937002C0A6
:1009800080E090E00E9423172BC1112321F08D2FCE
:100990009C2F937002C080E090E00E94391720C124
:1009A0008D2F112319F00E94A51202C00E9400137E
:1009B0000E94771315C18C2F837009F047C0111165
:1009C0000BC12D2F229526952770220F220F6D2FF8
:1009D0006F70862F90E0A0E0B0E0022E04C0880F78
:1009E000991FAA1FBB1F0A94D2F7D4FF10C04FE073
:1009F00050E060E070E004C0440F551F661F771F91
:100A00002A95D2F7409550956095709503C040E0C7
:100A100050E0BA01C695C695C3708A019B01082BA8
:100A2000192B2A2B3B2BC901B801C23049F058F4CD
:100A3000C13019F00E94E406CFC00E94D206CCC09B
:100A40000E94F606C9C00E94D006C6C0112319F044
:100A50008C2F817001C08695882309F4BDC02D2F8D
:100A6000229526952770220F220F6D2F6F70862FEB
:100A700090E0A0E0B0E0022E04C0880F991FAA1FEA
:100A8000BB1F0A94D2F7D4FF10C04FE050E060E0E3
:100A900070E004C0440F551F661F771F2A95D2F7D8
:100AA000409550956095709503C040E050E0BA01C4
:100AB000C695C695C3708A019B01082B192B2A2B5A
:100AC0003B2BC901B801C23049F058F4C13019F0CC
:100AD0000E94A90781C00E9497077EC00E94BB07A1
:100AE0007BC00E940A0778C0CF70112339F08C2F89
:100AF0000E9430078D2F0E94DB036EC08D2F0E9455
:100B0000E2038C2F0E94510767C0D23F21F128F4E5
:100B1000D03F41F0D13FC1F043C0D33F19F1D43FA2
:100B200079F03EC0112341F0053008F051C08C2F00
:100B30008F710E9476074CC0063008F049C0F7CF8D
:100B400080915B0282FF18C0112339F08C2F8F71C6
:100B50000E9430073DC01123C9F38C2F8F710E9472
:100B6000510736C0112329F08C2F8F710E941B076B
:100B70002FC00E9416072CC0112349F0CF718C2F73
:100B80000E94300763E08C2F0E94820C21C081E01C
:100B90000E949D0C0230E0F082E00E949D0C18C083
:100BA000112331F0002391F28D2F0E94A90210C071
:100BB000002399F2D93349F41FEF27EE33E01150A7
:100BC00020403040E1F700C000008D2F0E94530309
:100BD00088EF8C0D843020F40E94FE160E943E02A5
:100BE000DD20C9F00E94F00B80FD15C0F7011282D4
:100BF0000E94EA0B0E943007C7010E942C060E9447
:100C0000EA0BDF91CF911F910F91FF90EF90DF9052
:100C1000CF900C945107DF91CF911F910F91FF90CE
:100C2000EF90DF90CF9008950F931F93CF93DF93B2
:100C3000EC01688179818A810E9472088C010E948E
:100C4000CD070E94BE06B801CE010E94E903DF91E4
:100C5000CF911F910F910895CF93DF93EC0198816D
:100C600089812B813C81232B31F08F3F31F481E04E
:100C70009F3F19F403C081E001C080E080FD1DC0EA
:100C8000CE010E94DC01811110C00E94F40B882368
:100C9000A1F08A81882389F080915B0282FD0DC0DA
:100CA00082E0DF91CF910C949D0CCE010E9414063E
:100CB000CE01DF91CF910C94BD01DF91CF910895CA
:100CC00080E090E00E94231780E090E00E943917B6
:100CD0000E941B0C0E943D0C0E94A8140C947713D8
:100CE00080910201909103010E9495170C94600677
:100CF0000E940B0C0C94700692959F70963079F0C0
:100D000010F4925001C09A50923068F4803F69F01C
:100D100018F4883E40F409C0843F29F406C0883E98
:100D200020F0813F11F080E0089581E00895FC01FA
:100D3000808191810E9467080E947C060895CF936C
:100D4000DF9300D000D01F92CDB7DEB70F900F9089
:100D50000F900F900F90DF91CF910895CF93DF9375
:100D600000D000D000D0CDB7DEB726960FB6F894ED
:100D7000DEBF0FBECDBFDF91CF91089508950895D6
:100D80000C94BF060C94C0060E94C2066093C80172
:100D90007093C9018093CA019093CB010C946006B3
:100DA0000C94C4060F931F930091C8011091C901C0
:100DB0002091CA013091CB01602B712B822B932B98
:100DC0001F910F910C94C4060F931F930091C801BB
:100DD0001091C9012091CA013091CB016023712388
:100DE000822393231F910F910C94C4060F931F939A
:100DF0000091C8011091C9012091CA013091CB0125
:100E000060277127822793271F910F910C94C406A6
:100E10000C94BF060E9408076093C4017093C5013B
:100E20008093C6019093C7010C94600660E070E067
:100E3000CB010C940A070F931F9341E050E060E050
:100E400070E08A019B0104C0000F111F221F331F95
:100E50008A95D2F7C901B8011F910F910C940A0726
:100E60000F931F9341E050E060E070E004C0440F36
:100E7000551F661F771F8A95D2F78091C401909104
:100E8000C501A091C601B091C7018A019B01082B41
:100E9000192B2A2B3B2BC901B8011F910F910C94E0
:100EA0000A070F931F9341E050E060E070E004C038
:100EB000440F551F661F771F8A95D2F740955095AE
:100EC000609570958091C4019091C501A091C60173
:100ED000B091C7018A019B01082319232A233B23D0
:100EE000C901B8011F910F910C940A070F931F932A
:100EF00041E050E060E070E004C0440F551F661F01
:100F0000771F8A95D2F78091C4019091C501A09175
:100F1000C601B091C7018A019B01082719272A271A
:100F20003B27C901B8011F910F910C940A070F9339
:100F30001F930091C4011091C5012091C601309109
:100F4000C701602B712B822B932B1F910F910C9457
:100F50000A070F931F930091C4011091C5012091BE
:100F6000C6013091C70160237123822393231F910F
:100F70000F910C940A070F931F930091C4011091D5
:100F8000C5012091C6013091C701602771278227D2
:100F900093271F910F910C940A0708952AE0929FBE
:100FA000800D1124E82FE695E695E695877051E0CF
:100FB00001C0550F8A95EAF785E0E89FF0011124FA
:100FC000EE56FE4F20E030E070E04081CB01022E73
:100FD00002C0969587950A94E2F7817081958427DF
:100FE0008523842781932F5F3F4F2530310569F793
:100FF00008952AE0929F800D1124682F66956695CA
:101000006695982F977085E0689FB001112440E0A5
:1010100050E080E0FB01E40FF51FEE56FE4F20810B
:1010200030E0092E02C0369527950A94E2F7217028
:101030003327042E01C0220F0A94EAF7822B4F5F58
:101040005F4F4530510531F70895BF92CF92DF923F
:10105000EF92FF920F931F93CF93DF938C01C09079
:10106000C401D090C501E090C601F090C701809105
:10107000C8019091C901A091CA01B091CB01C82AC1
:10108000D92AEA2AFB2ACFE1D0E0D701C6010C2EEB
:1010900004C0B695A795979587950A94D2F780FDD9
:1010A00004C0219790F7B12C07C0BC2EB8018C2F3B
:1010B0000E949E0F0197A9F38B2DDF91CF911F9175
:1010C0000F91FF90EF90DF90CF90BF900895CF9356
:1010D000DF93EC010E942508BE010E949E0FDF9164
:1010E000CF9108951F93CF93DF93EB0190919101DE
:1010F000992321F0CB010E94670813C0882349F08F
:10110000CB010E942508182F682FCE010E94CE0720
:1011100004C0CB010E94F907182FBE01812F0E9445
:101120009E0FDF91CF911F9108951F93CF93DF936F
:10113000C091CC0116E08091CD01C81799F0D0E0A4
:101140001C9FF0011D9FF00D1124E253FE4F4081C2
:10115000518162817381848195810E94AE062196BE
:10116000C770E9CFDF91CF911F9108954091FE01A3
:101170005091FF0160910002709101028091020282
:10118000909103020C94AE062091CC019091CD0178
:1011900056E02917A9F030E0529FF001539FF00D5F
:1011A0001124E253FE4F7181761306C070817813CB
:1011B00003C07281741306C02F5F3F4F2770E9CFC1
:1011C00080E0089581E00895EF92FF920F931F93BE
:1011D000CF93DF938091030282958F7009F065C0F1
:1011E00080910002882309F460C08091CC01F090C6
:1011F000CD011091FE010091FF01609101027091FB
:10120000020291E01F3F09F090E0C0910001D091EF
:101210000101292F96E0E92E8F1509F446C06115CA
:10122000710521F00F3F21F030E003C031E001C033
:10123000322F90E030FD36C0E89EF001E99EF00DBF
:101240001124DF01A253BE4F11963C911197301328
:1012500029C03C91311326C012963C91129731114E
:1012600021C013964D915C911497461B570B4C1758
:101270005D07C0F4809103028F7080618093030248
:10128000ED52FE4F80818F70806180838EEF91E000
:101290000E942C06DF91CF911F910F91FF90EF904C
:1012A0000C94950801968770B7CFDF91CF911F916D
:1012B0000F91FF90EF9008958F929F92AF92BF92FF
:1012C000CF92DF92EF92FF920F931F93CF93DF9312
:1012D000CDB7DEB761970FB6F894DEBF0FBECDBFB6
:1012E0008C0185E0F801DE011D9601900D928A9532
:1012F000E1F7D8011296EC909091FE012091FF0148
:1013000040910102509102024115510531F02F3FE9
:1013100031F481E09F3F19F403C081E001C080E017
:1013200080FD7CC1F801C080D180838094808EEFE5
:10133000A82E81E0B82EF0900002B401641B750B5A
:101340004091000150910101FF2009F411C18091E9
:101350000302382F307F6417750708F0CBC03111B6
:101360008AC0D21214C0C91212C0FE2CE1100FC0E4
:101370008F708061809303020E94B608C5010E94AD
:101380002C0680910302D80115968C9361C18114BB
:10139000910439F0BFEFDB1206C081E0CB1203C02D
:1013A00003C081E001C080E080FD03C081E08E25A4
:1013B00002C080E090E080FF10C04E2D6D2D8C2D7E
:1013C0000E94C408882349F08EEF91E00E942C0609
:1013D000EEEFF1E086E0DF019DC0892839F0BFEF34
:1013E000DB1206C081E0CB1203C003C081E001C064
:1013F00080E080FD03C081E08E2502C080E090E0A7
:10140000E82FE170BE2E80FF2CC04E2D6D2D8C2D4F
:101410000E94C408F82E811124C0CD86DE868D85F9
:101420009E850E946708292F22952F70223018F080
:10143000243090F405C09F7059F0811109C008C193
:101440009F7031F0D80115969C91907F09F400C1EE
:10145000805E883008F4FCC0C8010E942C06FB2C7A
:10146000F7C0FE2CEE2009F4F3C0809103028160E6
:101470008093030254C0D21206C0C91204C0E11006
:1014800002C0F80199C0C8010E949706882361F143
:10149000EE2051F120910302822F82958F7090E00F
:1014A000029774F08091FE019091FF0198878F83DD
:1014B00019869B868A862C87CE0107960E942C0669
:1014C00086E0F801AEEFB1E001900D928A95E1F768
:1014D0000E94E4080E94B6080AC0D21611F1C801A1
:1014E0000E94970681112CC0C8010E942C06FF247F
:1014F000F394AEC03111F1CF782D998A888AA60174
:101500006E2D89890E949F068EEF91E00E942C0625
:1015100086E0D5011D928A95E9F70E94B608F12C64
:1015200097C0C912DCCFE110DACFF8018583C8017A
:101530000E942C0686E0D5011D928A95E9F788C0A5
:10154000EE2091F220910302822F82958F7090E01D
:1015500002970CF4B5CF8091FE019091FF019A8320
:1015600089831B829D828C822E83CE010196A6CF19
:101570006417750708F044C0FE2CEE2009F4B4CFC0
:10158000D21230C0C9122EC02091030220FD21C00A
:10159000822F82958F70482F50E041155105C9F078
:1015A000F80125834F30510541F08F5F982F9295B8
:1015B000907F822F8F70892B8583C8010E942C0613
:1015C00086E0F801AEEFB1E001900D928A95E1F767
:1015D0003DC086E0F801AEEFB1E001900D928A9532
:1015E000E1F736C0C8010E949706811169CF80914A
:1015F0000302816080930302C8010E942C0628C068
:10160000782D998A888AA6016E2D89890E949F0665
:1016100086E0D5011D928A95E9F718C0EE2009F4FD
:1016200063CFC8010E949706F82E882309F45CCF87
:1016300086E0F801AEEFB1E001900D928A95E1F7F6
:101640008EEF91E00E94A3020E94E4080E94B60877
:101650008F2D61960FB6F894DEBF0FBECDBFDF9120
:10166000CF911F910F91FF90EF90DF90CF90BF909F
:10167000AF909F908F9008951F93CF93DF93CDB736
:10168000DEB72C970FB6F894DEBF0FBECDBF4F83E9
:10169000588769877A878B879C87CE0107960E9437
:1016A0005C098823D1F09F8188852A853B85232B7F
:1016B00031F08F3F31F481E09F3F19F403C081E0A6
:1016C00001C080E080FD47C04F81588569857A85DB
:1016D0008B859C850E94AE063EC086E0FE01379653
:1016E000DE01119601900D928A95E1F7FF81E88560
:1016F0006A857B856115710531F0EF3F31F481E03A
:10170000FF3F19F403C081E001C080E080FD23C0E9
:101710002091CD0130E0C901019687709927409151
:10172000CC0150E084179507F1F1F983EA837D83BA
:101730006C8396E0929FD001939FB00D1124A25329
:10174000BE4FFE01319601900D929A95E1F780937C
:10175000CD010E94950816E08091CC019091CD01B9
:10176000891771F1189FC001112482539E4F0E9466
:101770005C09882329F1E091CC011E9FF00111241E
:10178000E253FE4F40815181628173818481958152
:101790000E94AE068091CC0190E001968770992757
:1017A0008093CC01D9CF0E9478061092CD0110927F
:1017B000CC01EEEFF1E086E0DF011D928A95E9F7BA
:1017C0002C960FB6F894DEBF0FBECDBFDF91CF9140
:1017D0001F91089580910C028595859585950895B2
:1017E00080910C028770089590910C02977081E0AF
:1017F00009F480E0089580911702089590911702EE
:10180000892B809317020895809590911702892360
:10181000809317020895109217020895909116026E
:10182000892B809316020895809590911602892342
:1018300080931602089510921602089580910D0269
:10184000089508950C94210C0C94220C90915B0245
:1018500092FD08C090910D02981721F080930D021F
:101860000C94240C089580910D02882329F0109285
:101870000D0280E00C94240C0895CF93DF93E09147
:101880000201F0910301809117028083E09102012F
:10189000F0910301908180911602892B80838091C1
:1018A0000D02882381F0E0910201F0910301908103
:1018B000892B808380910201909103010E944F1730
:1018C00081110E94330CC0910201D091030148E0C4
:1018D00050E064E072E0CE010E94901F892B69F015
:1018E00088E0FE01A4E0B2E001900D928A95E1F754
:1018F000CE01DF91CF910C940A17DF91CF9108951B
:101900000C94210C90915B0292FD10C098E0899F8D
:1019100090011124262B20930C020E943007809105
:101920000C028595859585950C94800C0C94300758
:1019300010920C0280E00C94800C20910C02809597
:10194000822380930C02982F977099F430E0482FEF
:10195000082E000C550B2417350759F090915B02A7
:1019600092FD07C08595859585950E9451070C9439
:10197000980C089590915B0292FB222720F928177A
:1019800069F080FB92F990935B0280915A029091EA
:101990005B020E94080D82E00C949D0C08958091DA
:1019A0005B0282FB882780F991E089270C94BA0CAE
:1019B00081E00C94BA0C80E00C94BA0C6FEF7FEFCE
:1019C00080E090E00C94C91F80E090E00E94A51F89
:1019D00021E0893E9E4F09F020E0822F089582E0A9
:1019E00090E00C949D1F83E090E00C949D1FCF939A
:1019F00084E090E00E949D1FC82F82E290E00E9448
:101A00009D1F2C2F30E0A901582BCA01CF910895BA
:101A1000CF93C92F682F84E090E00E94AB1F6C2FFA
:101A200082E290E0CF910C94AB1FAB01BC018FE040
:101A300090E00C94BD1FAB01BC0183E190E00C94DD
:101A4000BD1F60E070E0CB010C941B0D60E070E006
:101A5000CB010E94150D0C94210D69EE7EEF80E004
:101A600090E00E94C91F60E082E090E00E94AB1FFE
:101A700060E083E090E00E94AB1F1092C8011092DA
:101A8000C9011092CA011092CB0160E084E090E09D
:101A90000E94AB1F60E082E290E00E94AB1F60E01A
:101AA00085E090E00E94AB1F60E086E090E00E943D
:101AB000AB1F6FEF87E090E00E94AB1F40E050E06B
:101AC000BA0188E090E00E94BD1F60E08DE090E0E8
:101AD0000E94AB1F40E050E0BA0188E190E00E9414
:101AE000BD1F60E087E190E00E94AB1F40E050E046
:101AF000BA018CE190E00E94BD1F60E070E080E2DE
:101B000090E00E94C91F40E050E0BA0188E190E0F7
:101B10000E94BD1F0C94260D0C942D0D682F8EE095
:101B200090E00C94AB1F0E94441860932C027093B9
:101B30002D0280932E0290932F02609328027093BF
:101B4000290280932A0290932B02089585B780681A
:101B500085BF85B7806885BF089581E008950C949E
:101B6000AD0D08950C94B10D0C94B10D0C94B40D01
:101B70000C94B10D0C94B80D0C94B10D0E94A60DEF
:101B80008AE790E10E94F4160E94BC0D0C94BA0DF5
:101B90000E94B20D0C94B10D0E9494100C943D0261
:101BA0000E942F180E9479110E94CC0D0C94B60D42
:101BB0005F926F927F928F929F92AF92BF92CF92DD
:101BC000DF92EF92FF920F931F93CF93DF93CDB7E6
:101BD000DEB72A970FB6F894DEBF0FBECDBF0E94C6
:101BE0008E11C82E81110E94930D38E1832E32E0B0
:101BF000932E00E010E0502E802F0E94B8105C0160
:101C0000F401619071904F01682679266114710486
:101C1000B1F40F5F1F4F0830110569F78FEF89830B
:101C20008A831B820E9438188160782F9D838C8361
:101C300049815A816B818D810E9459023AC08091FD
:101C4000300281FD0E94C110D12CEE24E394F12CCE
:101C5000C3018E219F21892B29F10E94AF0D88237A
:101C6000A9F0DE825F82AE20BF2081E0AB2809F4BC
:101C700080E088870E9438188160782F9A8789874A
:101C80004E815F8168858A850E945902000F111F6D
:101C9000F801E85EFD4F80819181E826F926F18206
:101CA000E08207C0D394EE0CFF1CFAE0DF12D0CF25
:101CB000B0CF81E0C11001C080E02A960FB6F89441
:101CC000DEBF0FBECDBFDF91CF911F910F91FF906F
:101CD000EF90DF90CF90BF90AF909F908F907F90CC
:101CE0006F905F9008950E94D80D0E9495130C94F8
:101CF0004E02CF93DF930E94A30FEC01811521E5E3
:101D0000920708F045C0811530E5930708F094C0AC
:101D1000883E910528F5803E910508F0F8C0883A84
:101D2000910570F4853A910508F07CC081309105E9
:101D300009F475C008F4E8C0049708F0E8C0E4C0EE
:101D40008F3B910508F0E0C0C85AD0E0CC0FDD1FF2
:101D5000C65BDE4F0990D881C02DCE019464D8C0F7
:101D6000811540E2940758F4811551E0950708F079
:101D7000CEC08D3E910508F4C7C09065C9C0C1159D
:101D800080E4D80708F4C0C0DF70CE01906AC0C0FC
:101D9000811525E59207A8F4811534E5930708F02D
:101DA00095C0811543E5940708F07BC0811552E585
:101DB000950708F061C0D82FCC27CE01816F906ABB
:101DC000A7C0C11589E5D807A0F4C11528E5D20739
:101DD00008F082C0C11536E5D30708F095C08C2FF6
:101DE0000E9437108F7190E0D82FCC27CE019062DF
:101DF0008FC0C1154AE5D40708F474C0CE019056CF
:101E00008115904208F080C08D2F8F710E9437108D
:101E1000DD27D0628F71AE01582BCA0179C081E0F5
:101E200090E076C0C55AD0E0C858DE4F8881C82FF0
:101E3000D0E0CE0190646CC074E0969587957A9559
:101E4000E1F7282F23703C2F337081E090E002C02F
:101E5000880F991F3A95E2F79C68AC01522B9A01C2
:101E60009C2F9F709695969550E2959FE0011124C6
:101E7000C9018C2B9D2B4CC08370992721E030E049
:101E800002C0220F331F8A95E2F79C2F96959695F4
:101E900080E2989FE0011124C22BD32BCE019C68D5
:101EA00037C08370992721E030E002C0220F331F32
:101EB0008A95E2F79C2F9695969540E2949FE001D3
:101EC0001124C22BD32BCE019A6822C0D82FCC2745
:101ED000CE01846F906A1CC0DC2FCC27CE01806FAE
:101EE000906A16C08C2F8F700E94371094E0D695A0
:101EF000C7959A95E1F7CF70D0E0DC2FCC27D06959
:101F00009E01282BC90104C080E090E001C0CE01F1
:101F1000DF91CF91089520E5829FC0011124FC013B
:101F20002AE0729FE00DF11D1124E60FF11DEE0F66
:101F3000FF1FE852FF4F8591949108950E948B0FE7
:101F40000E94790E08958238910569F1B0F48133C9
:101F5000910509F46DC048F48932910509F463C014
:101F60008A32910509F469C008958533910509F411
:101F700055C089339105B9F00895833E910569F103
:101F800038F4803E9105B1F0823E910509F1089543
:101F9000863E9105A9F1873E9105B9F1843E9105F0
:101FA00009F064C023C020915A0220FD4FC021FDDA
:101FB0004DC0089580915A0280FD44C080915B021B
:101FC00080FF44C080915A0284FD42C083EE4DC020
:101FD00080915A0282FF38C0F5CF80915A0282FD6B
:101FE00033C080915B0280FD31C0ECCF80915B02F9
:101FF00081FF32C080915A0284FD2AC087EE35C02D
:1020000080915A0283FF26C0F5CF80915A0283FD4A
:1020100021C080915B0281FD1FC0ECCF80915A02EC
:1020200085FD1CC01DC080915A0285FD19C016C0D7
:1020300080915A0286FD16C017C080915A0286FD13
:1020400013C010C089E311C082EE0FC080EE0DC036
:1020500080E00BC086EE09C084EE07C089E205C0AF
:1020600085E303C08AE201C081E390E00895909186
:102070005A0292FF0DC0282F2871283019F4877F4B
:10208000846006C0282F2471243011F48B7F88606F
:1020900093FF0DC0282F2871283119F4877E8461A1
:1020A00006C0282F2471243111F48B7E8861209181
:1020B0005B0220FF0DC0382F3871383019F4877F4C
:1020C000816006C0382F3171313011F48E7F886005
:1020D00021FF0DC0282F2871283119F4877E8161D6
:1020E00006C0282F2171213111F48E7E886194FD64
:1020F000877E089580E008950C94DE0C0E948E1176
:102100008FE39CE90197F1F700C000000E948E1157
:1021100080E00E94B81080FF04C00E947C100C94E4
:10212000851808950C947E100E94E40C811102C061
:102130000E948C0D0E94EF0C809330020E94F70CDD
:1021400090935B0280935A020E9492100E94F30CBB
:10215000682F70E080E090E00E94D0066091C4019A
:102160007091C5018091C6019091C7010C94080738
:10217000E82FF0E0EE0FFF1FE459FD4F80819181C1
:102180000895089580EA8A95F1F7089500C00895AA
:102190000C94C21008950C94CA100C94CB100C949B
:1021A000CA100C94CF10F894E82FE295EF70F0E08D
:1021B00031A1282F2F7081E090E001C0880F2A956F
:1021C000EAF7982F9095932391A392A1892B82A34C
:1021D000789408950F931F93CF93DF93C5E8D1E0D0
:1021E00089918F3F11F00E94D31081E0CD38D8073C
:1021F000B9F7CBE7D1E005E811E089918F3F11F005
:102200000E94D3100C171D07C1F7DF91CF911F91CA
:102210000F910895BF92CF92DF92EF92FF920F93AA
:102220001F93CF93DF938C01C62FD0E0CE018B5745
:102230009E4F6C01FC0190819F3F09F450C0B62E67
:10224000F894E92FE295EF70F0E081A19F7021E012
:1022500030E001C0220F9A95EAF7822B81A382A178
:102260002095282322A378940E94C610EBE7F1E082
:1022700045E851E021E030E0E12CF12C61916F3F25
:1022800089F0A62FA295AF70B0E090968C9190E067
:102290006F7002C0959587956A95E2F780FD02C040
:1022A000C90102C080E090E0E82AF92A220F331F1A
:1022B0004E175F0719F7F60180818F3F11F00E94DA
:1022C000D31061E0E114F10409F460E08B2D0E9469
:1022D000C810CC0FDD1FC00FD11FF982E882DF913B
:1022E000CF911F910F91FF90EF90DF90CF90BF9013
:1022F00008950E94EA1080E1ECE6F2E0DF01982FF9
:102300001D929A95E9F7ECE5F2E0DF011D928A95BE
:10231000E9F788E00E94D9110C94C801FF920F934D
:102320001F93CF93DF93CDB7DEB760970FB6F894C6
:10233000DEBF0FBECDBF8E010F5F1F4F80E1F801E2
:1023400011928A95E9F7F12C6F2DC8010E940A11AC
:10235000F394F8E0FF12F8CF40E150E0B8018CE5CB
:1023600092E00E94901FFF24F394009709F4F12C4F
:10237000892B41F080E1F801ACE5B2E001900D92CB
:102380008A95E1F72F2D48E06CE672E08CE592E04B
:102390000E94DA110E94CA018F2D60960FB6F89440
:1023A000DEBF0FBECDBFDF91CF911F910F91FF9088
:1023B00008950895FF920F931F93CF93DF93F82E04
:1023C000092F162FD72FC42F222349F081E08093A5
:1023D00033020E9438189093320280933102809128
:1023E00033028823D9F080913102909132020E9409
:1023F0005018059798F0EF2DF02FA12FBD2F80E0FA
:1024000090E04C2F50E08417950734F421913191DE
:102410002D933D930196F7CF10923302DF91CF9128
:102420001F910F91FF9008950E94281A0E94D00DCD
:102430000C94341A0E94381A0E94730E0C94521A8B
:102440000E94D6170E940F1A0E94BE0D0E941412FD
:102450000E941A120E94C80DFBCF80913A0280FFA1
:1024600006C06091090170E0660F771F26C081FFEA
:1024700004C06091090184E005C082FF07C060913B
:10248000090188E0689FB001112417C090913902BA
:102490009923D1F060910801961788F720910901DE
:1024A00088E0289F90011124929FA001939F500DD6
:1024B000112470E0CA010E94621F6038710540F467
:1024C0006115710519F406C068E070E0862F089563
:1024D0008FE7089581E0089580913A0280FF08C057
:1024E0006091050170E0759567957595679521C0B8
:1024F00081FF06C06091050170E07595679519C070
:1025000082FF04C06091050170E010C09091380214
:10251000992399F0609104019617A0F78091050125
:10252000899FC001112470E00E94621F603871050C
:1025300040F46115710519F406C061E070E0862F62
:1025400008958FE7089581E008958D3E21F40E945B
:102550002D12819504C08E3E29F40E942D12809385
:102560003E0208958F3E21F40E942D12819504C0F1
:10257000803F29F40E942D1280933D020895893FE7
:1025800019F40E946C1205C08A3F31F40E946C124B
:10259000819580933F0208958B3F21F40E946C1235
:1025A000819504C08C3F29F40E946C1280934002F4
:1025B00008959FE0980F983078F421E030E0A90169
:1025C00002C0440F551F9A95E2F7CA0190913C0250
:1025D000892B80933C0208958D3F21F480913A022B
:1025E00081600BC08E3F21F480913A02826005C069
:1025F0008F3F29F480913A02846080933A020895D3
:102600008D3E39F490913E0297FF35C010923E0204
:1026100059C08E3E29F490913E021916BCF32BC08E
:1026200090913D028F3E29F497FF25C010923D0204
:1026300049C0803F19F41916CCF31DC090913F0298
:10264000893F29F41916BCF410923F023BC08A3F1F
:1026500019F497FF10C0F8CF8B3F39F490914002E6
:1026600097FF09C0109240022DC08C3F21F4909139
:1026700040021916BCF39FE0980F983080F421E0D7
:1026800030E0A90102C0440F551F9A95E2F7CA0134
:10269000809590913C02892380933C0213C08D3F2A
:1026A00021F480913A028E7F0BC08E3F21F48091FD
:1026B0003A028D7F05C08F3F29F480913A028B7FCB
:1026C00080933A0280913D02811106C080913E02C2
:1026D000811102C01092390280913F02811106C01F
:1026E00080914002811102C01092380208950E9428
:1026F000381820913D02211104C020913E0222236E
:1027000021F0909337028093360220913F022111ED
:1027100004C020914002222321F09093350280933F
:1027200034028BE392E00C941517EF92FF920F9313
:102730001F93CF93DF9300D000D000D0CDB7DEB78A
:1027400086E0EBE3F2E0DE01119601900D928A95AE
:10275000E1F7E0903D02F0903E0200913F021091BF
:10276000400210923D0210923E0210923F021092DF
:102770004002E11003C0FF2009F45DC080913602E1
:10278000909137020E945018AC0190913902992320
:1027900039F020910A0130E02417350758F04BC07A
:1027A00020910B018AE0289F9001112424173507FE
:1027B00018F041C09F3F19F09F5F90933902EE20BF
:1027C00061F00E942D121E1414F09FEF01C091E0E1
:1027D000989F902D112490933D02FF2061F00E945C
:1027E0002D121F1414F09FEF01C091E0989F902DBF
:1027F000112490933E0230913D023323E1F0209169
:102800003E022223C1F045EB3403C0011124992379
:1028100019F090933D0203C081E080933D0235EBB7
:102820002303C0011124992319F090933E0203C0A1
:1028300081E080933E02011103C0112309F45DC0C1
:1028400080913402909135020E945018AC01909111
:102850003802992339F02091060130E0241735071A
:1028600058F04BC0209107018AE0289F9001112465
:102870002417350718F041C09F3F19F09F5F9093D0
:102880003802002361F00E946C12101614F09FEFC2
:1028900001C091E0989F902D112490933F02112345
:1028A00061F00E946C12111614F09FEF01C091E0CC
:1028B000989F902D11249093400230913F02332332
:1028C000E1F0209140022223C1F045EB3403C00126
:1028D0001124992319F090933F0203C081E0809363
:1028E0003F0235EB2303C0011124992319F0909383
:1028F000400203C081E08093400280913D0281113B
:102900000BC080913E02811107C080913F0281116E
:1029100003C08091400281110E947713EB82FC82F8
:102920000D831E8386E0FE013196ABE3B2E0019099
:102930000D928A95E1F726960FB6F894DEBF0FBE8A
:10294000CDBFDF91CF911F910F91FF90EF90089530
:10295000EBE3F2E086E0DF011D928A95E9F7109241
:1029600039021092380210923A020895CF93DF9301
:10297000EC01FB018281882309F43CC1C430FDE5F0
:10298000DF0760F4CB3F9CE5D90788F49E01225015
:102990003C452431310508F02EC109C0C236EDE5B1
:1029A000DE0729F0C63AFDE5DF0709F024C10E94E1
:1029B000F70C90935B0280935A02C1318CE5D807E3
:1029C00009F4C6C008F042C0C930ECE5DE0709F4DE
:1029D0009BC000F5C5308CE5D80709F485C078F4B4
:1029E000C330ECE5DE0709F478C008F07AC0C230E5
:1029F000DC4509F0F5C080915A028160EFC0C73014
:102A00009CE5D90709F478C008F07AC080915A0291
:102A10008061E4C0CD30FCE5DF0709F487C058F4DD
:102A2000CB309CE5D90709F479C008F07BC08091D0
:102A30005A0288606FC0CF30FCE5DF0709F480C020
:102A400008F082C080915A02877FC8C0CE3F9CE5C3
:102A5000D90709F471C000F5C531FCE5DF0709F4B9
:102A600085C068F4C3319CE5D90709F475C008F046
:102A700095C00E94780680915A028F77AFC0CC3FF4
:102A8000FCE5DF07A9F108F054C0CB3FDC4509F0B5
:102A9000A7C080915B0240C0C230EDE5DE0709F4BB
:102AA00089C058F4C1158DE5D80709F45AC008F05B
:102AB00069C080915B0282602FC0C236EDE5DE07FF
:102AC00009F47CC0C63AFDE5DF0709F481C0C330D4
:102AD000DD4509F085C080E06EC080915A028260B9
:102AE0007DC080915A0216C080915A02886076C0DB
:102AF00080915B0282604FC080915A0280626EC0FA
:102B000080915A0280646AC00E94780680915A02BD
:102B1000806864C0846062C081603DC080915A0258
:102B20008E7F5CC080915A028D7F58C080915A027E
:102B300016C080915B0218C080915B028D7F2BC014
:102B400080915A028F7E4AC080915A028F7D46C082
:102B500080915A028F7B42C080915A02877F8B7F7F
:102B60003DC080915B028D7F8E7F15C080915A029F
:102B700082FB222720F991E0922790FB82F990FBBB
:102B800083F92CC080915B02982F909591708E7F75
:102B9000892B90FB81F980935B0222C00E9478060A
:102BA00080915A0287FB222720F991E0922790FB1F
:102BB00087F914C081E00E948E0D12C080915A02E4
:102BC00084FB222720F991E0922790FB84F906C02C
:102BD00080915A02982F909590FB80F980935A0229
:102BE00080915A0290915B020E94080D0E94780623
:102BF00080E001C081E0DF91CF910895CF93DF9312
:102C000086319C4541F5EB010E94FB0B982F8A8190
:102C10002091020130910301882379F09A7A81E0B2
:102C200009F480E080934102911102C069E201C081
:102C300065E3C9010E9491170AC080914102811188
:102C400002C069E201C065E3C9010E9493170E94B6
:102C50003D0C80E001C081E0DF91CF9108950F939A
:102C60001F93CF93DF93C42FD22FFC01828188233F
:102C7000C9F0409344020E94381890934302809315
:102C8000420280E28C0F883008F057C0C77081E0A4
:102C900001C0880FCA95EAF7DF91CF911F910F917C
:102CA0000C94DB0380914402481330C080914202AF
:102CB000909143020E945018883C910538F510E22B
:102CC0001D0FCD17B9F080E28C0F883040F4C7702B
:102CD00081E001C0880FCA95EAF70E94E20318302C
:102CE00028F581E09D2F977001C0880F9A95EAF72B
:102CF0000E94DB03802F0E94D2031830F0F4D770BB
:102D000081E001C0880FDA95EAF70AC080E28C0FF3
:102D1000883098F4C77081E001C0880FCA95EAF73F
:102D2000DF91CF911F910F910C94E203802FDF91DF
:102D3000CF911F910F910C94D203DF91CF911F91EE
:102D40000F9108950F939C01CB01243F4CE534076C
:102D500031F188F4293DFCE53F07D9F02A3D4CE5E7
:102D6000340779F1283D3C45A9F506E221EE41EE14
:102D700068ED7CE52BC0263FFCE53F07E1F0A8F0BD
:102D8000273F3C4539F507E225EE46EE67EF7CE547
:102D90001DC007E225EE45EE69ED7CE517C006E2B1
:102DA00021EE40EE64EF7CE511C007E225EE44EE33
:102DB00065EF7CE50BC006E221EE42EE66EF7CE5B6
:102DC00005C008E221E045EE6AED7CE50E942F1681
:102DD00080E008C0FC018281882319F0109244022F
:102DE00001C081E00F91089590938F0180938E012F
:102DF000089590934A02809349020895E091490210
:102E0000F0914A02309721F00190F081E02D099471
:102E100080E00895E0914902F0914A02309721F054
:102E20000280F381E02D09940895E0914902F09128
:102E30004A02309739F022E0DC012C930480F581BE
:102E4000E02D0994089520914702309148022817F7
:102E5000390771F09093480280934702E09149024C
:102E6000F0914A02309721F00680F781E02D099415
:102E7000089520914502309146022817390771F0D4
:102E80009093460280934502E0914902F0914A02F4
:102E9000309721F00084F185E02D09940895FC011C
:102EA000329697E080E0915029F021912223D9F3C6
:102EB0008F5FF9CF0895662349F0FC01329608969A
:102EC0002191621729F0E817F907D1F780E00895FA
:102ED00081E008959C01FC0132969FEF80E04191D2
:102EE000461789F09F3F19F4411101C0982F8F5F59
:102EF0008630A9F79F3F39F0F901E90FF11D97FDE1
:102F0000FA956283089508959C012A5F3F4FFC0162
:102F10004281461301C01282019682179307B9F7C6
:102F200008950C946A170C948417029626E0FC010D
:102F300011922A95E9F7089508950C949C1783E05F
:102F400080934B020C949D17811102C081E001C057
:102F500082E080934B020C949D170C94A41781E09F
:102F600080934B020C949D170C94AF1708950C940A
:102F7000B6170C94B7170C94B6170C94B6170C949C
:102F8000B617CF930E94BD170E948E110E94BB17E7
:102F9000C0E08C2F0E94B810892B29F4CF5FC83075
:102FA000C1F780E001C081E0CF91089508951F929C
:102FB0000F920FB60F9211248F939F93AF93BF93ED
:102FC00080914C02811113C080917C0290917D020E
:102FD000A0917E02B0917F024196A11DB11D809308
:102FE0007C0290937D02A0937E02B0937F02BF91FA
:102FF000AF919F918F910F900FBE0F901F901895DA
:1030000080918402843031F10E942E0210924C0291
:1030100020E488E190E00FB6F894A89580936000D2
:103020000FBE2093600083B7817F846083BF83B726
:10303000816083BF7894889583B78E7F83BF0FB6F6
:10304000F894A89580916000886180936000109248
:1030500060000FBE08950E9478060C94320282E050
:1030600084BD93E095BD9AEF97BD80936E0008955F
:103070002FB7F89480917C0290917D02A0917E02FE
:10308000B0917F022FBF08952FB7F89460917C0212
:1030900070917D0280917E0290917F022FBF0895F2
:1030A0009C014FB7F89480917C0290917D02A09191
:1030B0007E02B0917F024FBF821B930B08957894DC
:1030C0001F920F920FB60F9211248F939F93AF937D
:1030D000BF9380917C0290917D02A0917E02B0917D
:1030E0007F020196A11DB11D80937C0290937D0209
:1030F000A0937E02B0937F02BF91AF919F918F9179
:103100000F900FBE0F901F90189587E797E7909349
:103110000108809300089AE088E10FB6F894A8951A
:10312000809360000FBE90936000FFCF80915802A3
:103130000895089522E02093E9002FEF3091E800F0
:10314000215035FD06C035ED3A95F1F7000021110B
:10315000F5CF2091E80025FF0BC040E050E066E08D
:1031600070E00E94C41A8091E8008E778093E80096
:103170000895CF93DF9321E02093E9002FEF309162
:10318000E800215035FD06C035ED3A95F1F7000015
:103190002111F5CF2091E80025FF14C0EC0140E09B
:1031A00050E068E070E00E94C41A8091E8008E77D9
:1031B0008093E80088E0FE01A0E5B2E001900D9266
:1031C0008A95E1F7DF91CF91089580934D02709336
:1031D0004F0260934E0280918402843001F582E0B8
:1031E0008093E9008FEF9091E800815095FD06C033
:1031F00095ED9A95F1F700008111F5CF8091E800E7
:1032000085FF0DC040E050E063E070E08DE492E0A7
:103210000E94C41A8091E8008E778093E800089598
:10322000BC0184E00C94E518BC0183E00C94E51823
:1032300080918302811109C00E94551C0E94B21C1A
:103240008091E20084608093E200089510928302EE
:1032500008950C94B4176091800281E0611101C05F
:1032600080E00C949F179091840281E0943009F0E3
:1032700080E0609180020C94A41742E061EC81E050
:103280000E94CE1B42E261EC82E00E94CE1B909134
:10329000840281E0943009F080E0609180020C9417
:1032A000AD1780918602833009F461C030F481301B
:1032B00071F0823009F49AC008958A3009F486C00A
:1032C0008B3009F46CC0893009F0A8C020C080910F
:1032D0008502813A09F0A2C08091E800877F80933F
:1032E000E8008091890290918A02892B21F468E09C
:1032F00080E592E003C060E080E090E070E00E9432
:103300000F1B8091E8008B778093E80008958091EF
:103310008502813209F082C08091890290918A02EF
:10332000029708F07BC08091E800877F8093E800D7
:103330008091E80082FD05C0809184028111F8CF60
:103340006DC02091F3008091F20090E0922B0297E3
:1033500031F48091F100813011F0863021F48091B8
:10336000F100809358028091E8008B7753C08091E0
:103370008502813A09F052C08091890290918A02B7
:10338000892B09F04BC08091E800877F8093E8008B
:103390008091E80080FFFCCF8091180136C08091B9
:1033A00085028132D9F58091890290918A02892B18
:1033B000A9F58091E800877F8093E8000E94031CB4
:1033C00080918702809318010C9478068091850281
:1033D000813221F58091E800877F8093E8000E9488
:1033E000031C809188028093590208958091850280
:1033F000813AA1F48091E800877F8093E800809172
:10340000E80080FFFCCF809159028093F100809109
:10341000E8008E778093E8000C94031C089584B72D
:10342000877F84BF0FB6F894A8958091600088616B
:1034300080936000109260000FBE90E080E80FB6AD
:10344000F89480936100909361000FBE0C94AF17C5
:103450000E94551C0E94B21CE2EEF0E08081846064
:10346000808378940C94471F8CE091E00C94F916BB
:10347000809184028530A9F480918402853079F4AA
:103480000E940018809182028823B1F30E94C11724
:10349000882391F30E94AE1A0E947806EDCF0C9417
:1034A0002B18089508950C94551A292F332723308B
:1034B0003105C9F060F42130310581F02230310549
:1034C00009F044C08BE390E026EA31E043C02132AA
:1034D0003105E1F02232310549F138C082E190E056
:1034E00021EE31E037C099278130910549F028F06D
:1034F000029761F5E8E7F1E005C0E2EAF1E002C019
:10350000E6E8F1E0849190E09F0124C06115710527
:1035100041F061307105D1F489E090E021ED31E0B6
:1035200019C089E090E028EB31E014C06115710505
:1035300041F06130710551F48BE790E023EF31E009
:1035400009C080E490E02EE632E004C080E090E024
:1035500020E030E0FA0131832083089580E189BDC5
:1035600082E189BD09B400FEFDCF8091D8008F7D36
:103570008093D8008091E00082608093E000809189
:10358000E00081FDFCCF0895CF92DF92EF92FF9291
:103590000F931F93CF93DF93EC018B017A010E946D
:1035A000221C811133C0E114F10439F0F70180814C
:1035B0009181081B190BC80FD91FC12CD12C0115E3
:1035C000110519F18091E80085FD16C08091E80091
:1035D0008E778093E800E114F10449F0F7018081CF
:1035E0009181C80ED91ED182C08285E00FC00E9491
:1035F000221C882321F30AC089918093F100015095
:103600001109FFEFCF1ADF0ADACF80E0DF91CF9107
:103610001F910F91FF90EF90DF90CF900895209130
:103620008B0230918C022617370748F0611571051F
:1036300039F42091E8002E772093E80001C0B90109
:10364000FC0120E06115710579F1809184028823E5
:10365000F1F18530F1F18091E80083FD3CC080916B
:10366000E80082FD2EC08091E80080FFEBCF209122
:10367000F3008091F20090E0922B6115710551F0FA
:103680008830910538F421912093F100615071093F
:103690000196F3CF21E0089709F020E08091E8003F
:1036A0008E778093E800CECF2111CFCF0AC08091D2
:1036B0008402882361F0853061F08091E80083FD09
:1036C0000AC08091E80082FFF2CF80E0089582E096
:1036D000089583E0089581E0089520918B02309150
:1036E0008C022617370748F06115710539F42091CF
:1036F000E8002E772093E80001C0B901FC0120E02A
:103700006115710591F180918402882309F440C00C
:10371000853009F43FC08091E80083FD3DC0809171
:10372000E80082FD2FC08091E80080FFE9CF209162
:10373000F3008091F20090E0922B6115710559F031
:103740008830910540F424912093F1003196615026
:1037500071090196F2CF21E0089709F020E08091ED
:10376000E8008E778093E800CBCF2111CCCF0AC040
:1037700080918402882361F0853061F08091E800B7
:1037800083FD0AC08091E80082FFF2CF80E00895B7
:1037900082E0089583E0089581E00895982F97309E
:1037A00068F59093E900981739F07091EC0020913A
:1037B000ED005091F00003C0242F762F50E021FD42
:1037C00002C09F5FECCF3091EB003E7F3093EB0067
:1037D0003091ED003D7F3093ED003091EB00316092
:1037E0003093EB007093EC002093ED005093F000C9
:1037F0002091EE0027FDE5CF80E008958F70809343
:10380000E90081E008958091850287FF11C08091D1
:10381000E80082FD05C0809184028111F8CF11C0BB
:103820008091E8008B770BC080918402882349F057
:103830008091E80080FFF8CF8091E8008E77809338
:10384000E80008952091E4003091E50095E640916C
:10385000EC00842F817040FF23C08091E80080FD40
:103860001DC080918402882399F0853099F0809161
:10387000EB0085FD11C04091E4005091E500241754
:10388000350729F3915011F09A01E1CF84E00895B2
:1038900082E0089583E0089581E0089580E008952E
:1038A0004091E80042FFDDCF08950E94C31C0E94B2
:1038B000CB1CE0EEF0E0808181608083E8EDF0E0F9
:1038C00080818F77808319BCA7EDB0E08C918E7FCB
:1038D0008C9380818F7E80831092830208950F9352
:1038E0001F93CF93DF930E94C31C0E94CB1CC8ED93
:1038F000D0E088818F7788838881806888838881F9
:103900008F7D888319BC10928402109280021092DD
:1039100082021092810200EE10E0F80180818B7F1C
:10392000808388818160888342E060E080E00E943B
:10393000CE1BE1EEF0E080818E7F8083E2EEF0E04E
:10394000808181608083808188608083F8018081AC
:103950008E7F8083888180618883DF91CF911F91E2
:103960000F910895E8EDF0E080818F7E8083E7ED90
:10397000F0E080818160808384E082BF81E0809379
:1039800083020C946F1CE8EDF0E080818E7F8083D1
:103990001092E20008951092DA001092E10008956A
:1039A0001F920F920FB60F9211242F933F934F93B4
:1039B0005F936F937F938F939F93AF93BF93EF9397
:1039C000FF938091E10082FF0BC08091E20082FFB3
:1039D00007C08091E1008B7F8093E1000E94461F29
:1039E0008091DA0080FF1FC08091D80080FF1BC04B
:1039F0008091DA008E7F8093DA008091D90080FF79
:103A00000DC080E189BD82E189BD09B400FEFDCF12
:103A100081E0809384020E94181905C019BC10929D
:103A200084020E9426198091E10080FF19C08091D4
:103A3000E20080FF15C08091E2008E7F8093E2005B
:103A40008091E20080618093E2008091D8008062E2
:103A50008093D80019BC85E0809384020E942B19C2
:103A60008091E10084FF30C08091E20084FF2CC08F
:103A700080E189BD82E189BD09B400FEFDCF80915E
:103A8000D8008F7D8093D8008091E1008F7E809355
:103A9000E1008091E2008F7E8093E2008091E2005D
:103AA00081608093E20080918002882311F084E09D
:103AB00007C08091E30087FD02C081E001C083E080
:103AC000809384020E9433198091E10083FF29C012
:103AD0008091E20083FF25C08091E100877F809381
:103AE000E10082E080938402109280028091E100E4
:103AF0008E7F8093E1008091E2008E7F8093E200D0
:103B00008091E20080618093E20042E060E080E02A
:103B10000E94CE1B8091F00088608093F0000E948C
:103B20002919FF91EF91BF91AF919F918F917F9153
:103B30006F915F914F913F912F910F900FBE0F901A
:103B40001F9018951F920F920FB60F9211242F936A
:103B50003F934F935F936F937F938F939F93AF9315
:103B6000BF93CF93DF93EF93FF93C091E900CF70A2
:103B70008091EC00D82FD17080FDD0E81092E90040
:103B80008091F000877F8093F00078940E94E61D7A
:103B90001092E9008091F00088608093F000CD2BB6
:103BA000CF70C093E900FF91EF91DF91CF91BF916A
:103BB000AF919F918F917F916F915F914F913F91C5
:103BC0002F910F900FBE0F901F9018951F93CF93BA
:103BD000DF93CDB7DEB7AA970FB6F894DEBF0FBE5E
:103BE000CDBFE5E8F2E08091F100819322E0ED386D
:103BF000F207C9F70E9451198091E80083FF2EC196
:103C00008091850290918602492F50E04A305105FB
:103C100008F024C1FA01EE59FF4F0C94761F80384A
:103C200021F0823809F01AC108C080918102909178
:103C30008202992389F082600FC0809189028F707F
:103C4000873008F00BC18093E9008091EB0085FB81
:103C5000882780F91092E9009091E800977F90936F
:103C6000E8008093F1001092F100D1C0282F2D7F41
:103C700009F0F4C0882319F0823061F0EFC0809120
:103C80008702813009F0EAC0933009F080E0809328
:103C900082022EC08091870281112AC08091890200
:103CA0008F702FEF280F263008F0D8C08093E900DE
:103CB0002091EB0020FF1CC0933021F48091EB0099
:103CC000806214C09091EB0090619093EB0021E032
:103CD00030E0A90102C0440F551F8A95E2F74093D6
:103CE000EA001092EA008091EB0088608093EB007C
:103CF0001092E9008091E800877F8093E8000E949D
:103D0000031CACC08111AAC0109187021F7780915B
:103D1000E3008078812B8093E3008091E800877F27
:103D20008093E8000E94031C8091E80080FFFCCF94
:103D30008091E30080688093E300111102C082E06B
:103D400001C083E08093840289C08058823008F0EB
:103D500085C080918702909188028C3D53E0950741
:103D600079F583E08A838AE289834FB7F894DE018C
:103D7000139620E03EE051E2E32FF0E0509357002D
:103D8000E49120FF03C0E295EF703F5FEF708E2F4C
:103D900090E0EA3010F0C79601C0C0968D939D93D5
:103DA0002F5F243149F74FBF8091E800877F8093D0
:103DB000E8006AE270E0CE0101960E940F1B16C077
:103DC0006091890270918A02AE014F5F5F4F0E943D
:103DD000531ABC01892B09F441C09091E800977FE8
:103DE0009093E80089819A810E946D1B8091E80080
:103DF0008B778093E80032C0803881F58091E800AD
:103E0000877F8093E800809180028093F100809109
:103E1000E8008E7772CF811121C080918702909146
:103E2000880299270297D4F48091E800877F8093D5
:103E3000E80080918702809380020E94031C809199
:103E40008002811106C08091E30087FD02C081E0FD
:103E500001C084E0809384020E943D198091E800B3
:103E600083FF0AC08091E800877F8093E8008091FB
:103E7000EB0080628093EB00AA960FB6F894DEBF49
:103E80000FBECDBFDF91CF911F9108950895CF93BD
:103E9000809184028823A1F0C091E900CF709091B5
:103EA000EC00892F817090FD80E8C82B1092E9000A
:103EB0008091E80083FD0E94E61DCF70C093E90069
:103EC000CF91089597FB072E16F4009407D077FD45
:103ED00009D00E947C1F07FC05D03EF49095819587
:103EE0009F4F0895709561957F4F0895EE0FFF1FC6
:103EF0000590F491E02D0994AA1BBB1B51E107C06A
:103F0000AA1FBB1FA617B70710F0A61BB70B881F69
:103F1000991F5A95A9F780959095BC01CD010895F8
:103F2000FB01DC0104C08D910190801921F4415006
:103F30005040C8F7881B990B0895F999FECF92BDA0
:103F400081BDF89A992780B50895A8E1B0E042E0D4
:103F500050E00C94D11F262FF999FECF92BD81BD60
:103F6000F89A019700B4021639F01FBA20BD0FB6B7
:103F7000F894FA9AF99A0FBE08950396272F0E9493
:103F8000AC1F0E94AB1F252F0E94AC1F242F0C9446
:103F9000AC1F0196272F0E94AC1F0C94AB1FDC01B5
:103FA000CB01FC01F999FECF06C0F2BDE1BDF89A44
:103FB000319600B40D9241505040B8F70895F894EE
:023FC000FFCF31
:103FC200C8000E02280850011E0A14019618B918DA
:103FD2009A1814191019991801E200E900EA00B5BB
:103FE20000B600B700CD008301CC008A0192019493
:103FF200012102230224022502260227022A02B3F9
:1040020000B4006F007000818283E200E900EA00E0
:10401200B500B600B700CD008301CC008A01920141
:1040220094012102230224022502260227022A02E7
:10403200B300B4006F00700081828336323331F7EF
:0E404200C697669094F4F5F63593929134008B
:00000001FF
